:10000000280C06005F0C0200170C26006B001B0971
:100010006606130A020C8B000306240A6B00FF0C11
:10002000060026020300AC024306AB02FF0C8B0065
:100030004306340A070A050C8A004306210AAA026D
:100040000008000C2A000008490927002600400982
:100050004009400940094009400940094009400958
:100060006B00170C2600070A070226004009170C30
:10007000260040096606340A6B00170C2600070AA2
:10008000FF0C2900FF0C2800E802440AE902420A9A
:100090000008000C8A0043061308010C8A0043067E
:1000A0000708020C8A0043060308030C8A00430673
:1000B0000608040C8A0043060208050C8A00430661
:0200C000040832
:00000001FF
